:020000040000fa
:08000000a60604000000000048
:020000040000fa
:020000040002f8
:04afe000dfff00008f
:020000040000fa
:020000040002f8
:04afe400ffff00006b
:020000040000fa
:020000040002f8
:04afe80078ff0000ee
:020000040000fa
:020000040002f8
:04afec007dff0000e5
:020000040000fa
:020000040002f8
:04aff00078ff0000e6
:020000040000fa
:1000080000000000000000000000000000000000e8
:100018009e06000000000000000000000000000034
:10002800000000000000000000000000080a0000b6
:1000380000000000000000000000000000000000b8
:100048006a0a00000000000000000000f20a000038
:100058005e0b00008a0b000000000000000000009a
:100068000000000000000000000000000000000088
:100078000000000000000000000000000000000078
:10008800000000000000000000000000960a0000c8
:10009800c40a00000000000000000000000000008a
:1000a8000000000000000000000000000000000048
:1000b8000000000000000000000000000000000038
:1000c8000000000000000000000000000000000028
:1000d8000000000000000000000000000000000018
:1000e8000000000000000000000000000000000008
:1000f80000000000000000000000000000000000f8
:1001080000000000000000000000000000000000e7
:1001180000000000000000000000000000000000d7
:10012800000000002a0b0000000000000000000092
:1001380000000000000000000000000000000000b7
:1001480000000000000000000000000000000000a7
:100158000000000000000000000000000000000097
:100168000000000000000000000000000000000087
:100178000000000000000000000000000000000077
:100188000000000000000000000000000000000067
:100198000000000000000000b80b0000e40b0000a5
:1001a800100c00000000000000000000000000002b
:1001b8000000000000000000000000000000000037
:1001c8000000000000000000000000000000000027
:1001d8000000000000000000000000000000000017
:1001e8000000000000000000000000000000000007
:1001f80000000000000000000000000000000000f7
:1002080000000000000000000000000000000000e6
:1002180000000000000000000000000000000000d6
:1002280000000000000000000000000000000000c6
:1002380000000000000000000000000000000000b6
:1002480000000000000000000000000000000000a6
:100258000000000000000000000000000000000096
:100268000000000000000000000000000000000086
:0c0278000000000000000000000000007a
:020000040000fa
:10040000803e2000030007008100e900fcff3a0065
:1004100000000600831f7800c20320000400bc0017
:1004200066015100e0815900f23fb1000380b10044
:1004300006003500ee03090000000000423fb10055
:100440000380b100fbff3d001200b000223fb0006e
:10045000020035000280090000000000cf01780092
:10046000000006000001eb00869fbe00889fbe00d2
:100470008a9fbe008c9fbe00820578000004be00eb
:10048000e20107000800be006420e1000700390017
:1004900002003a00f1ff2f00f0ff27000160a000ea
:1004a00012022000f2908800560037006120e1001f
:1004b00003003a000b00a70001f8230051003700a9
:1004c00001f0a10002002100936424005200070003
:1004d0000800be0005003500b2fd2000930c24008a
:1004e00004002000690007000004be000005eb00c6
:1004f0000b00a6004f0dde0001f0a1000004be00bd
:1005000032982f0023ea23000f0107000001eb00bf
:10051000030020000b00a70003f82300ac00070035
:100520003e0107000000a7000a00a20082010700a8
:100530000b00e000030032000200200003f0230063
:10054000a200070001f0a2000006be000200200089
:1005500093042400fc0007000801be009c00070073
:10056000809fbe000c00be0022a22a00d3a7230059
:10057000f50007004f01be00950007000004be0013
:1005800001f0a100020020000398230022000700d0
:100590000800be00190035000001be00ea00070097
:1005a0000006be00b2c52900e3622300e600070092
:1005b00022222b00f3942b00850007000c01be00c3
:1005c000e1000700e273280083c0230080000700d9
:1005d0000c01be00dc00070042aa2a00a3e22b00a7
:1005e0007b0007000c01be00d70007000801be0019
:1005f000d50007000801be00750007000a00a7002b
:1006000001f0a2004f06be004f05be004f04be0021
:100610004f03be000000060014002000889fbe00ab
:100620008a9fbe00841f7800700107004f00780089
:1006300011003300f0ff2f00838f6c0006003b0099
:10064000040565000a00a7000800370009f0a600ad
:100650001000200008003700820f5400838f5c00d8
:10066000030039001000200001003e0000002000bf
:1006700009f0a7000000ea004f05be004f04be00cd
:100680000000e0000000060014002000869fbe006d
:10069000889fbe008a9fbe008c9fbe004f26dd0053
:1006a00052010700940133006120e1004300320051
:1006b0006250e10041003e003e0039006420e1004c
:1006c0003c003200058255000f003b000402e800a8
:1006d00038003a00800f5300818f5b0035003400f2
:1006e0000800be0003f0a10001f0a60003f0a00086
:1006f0000cf0a7003600070088013700060343000e
:1007000087834b000c4646000005530081855b0043
:10071000020033000a03be000c00a0000402e9003e
:10072000f6ff3b00850578000602430087824b00f8
:1007300004003a006000b80009f0a70001f0a00032
:10074000760137000002520081825a000704e0005f
:10075000040033000603430087834b008b05e90048
:10076000faff3700090578000604be000203be0048
:100770006011b8003a010700e00f5200e08f5a0004
:100780000700350002003c000c08a3000400320002
:100790000601be0003f0a0000cf0a7000c0007004b
:1007a0000a85680001f0a1000af0a70001f0a0008e
:1007b0005a0137000800be0058013700100220001f
:1007c0000cf0a600f09088005901370003f0a20059
:1007d000869fbe00889fbe008a9fbe008c9fbe0081
:1007e00002010700440133006450e1004f00320071
:1007f0006420e1005200320003826c0007003b00dd
:100800000905d0000306d000820f54000c065d00dd
:1008100002003900020032008901780003067800e6
:100820008582550004003d000003fd008103fd00aa
:100830008502ea008b854200840f720002003b00b3
:1008400060001000e08018006011b8000005eb00a7
:100850007a28e1000a00390006007800c75ddd0053
:10086000f707b200878075002d0037008281710084
:100870000a017800610560008180d1000080d3000a
:100880008502e900f9ff3b00060440008784480028
:1008900002003b0060041400e0841c000988a300ef
:1008a000070032008a817100828171006101640059
:1008b0008904d1000884d3008b05e80017003700b5
:1008c0000978a30013003a000b00e0001300340085
:1008d0008b05e9000804440089844c000a44740034
:1008e0000978a3000d003a000b00e0000700340077
:1008f0008b05e9000804440089844c0001003a009b
:100900000b0020000978a300f7ff32000001eb0084
:1009100002003700828171000a017800d0000700d0
:100920000cf0a70001f0a000fc0037006420e100fb
:1009300002003a00838f6c00fd0033000801be0006
:100940000200be00f5003700869fbe00889fbe00f3
:100950008a9fbe008c9fbe00a4000700e600330003
:1009600003866c006450e100240032006420e10042
:10097000270032006150e100220032006120e100d6
:10098000210032008b854200eb07b1000134b80032
:10099000003ab8000804420089844a00013ab800cd
:1009a0000030b8008880400009014a00040033008c
:1009b0000000400081804800020149008b05e900e9
:1009c000c909dd008301700001003200130020001e
:1009d000c814de004814dd004709de001200b20032
:1009e000c808de00088470009d00070001f0a10027
:1009f0000cf0a70001f0a000c80037006120e10062
:100a0000cb0032000801be000200be00f7ff370035
:100a10006150e100fcff3a00c5003700829fbe0034
:100a20000001be00790007000470a70003f0a100d8
:100a30006509b100180032000e0035006828e10099
:100a400007003500f0ff2f00f1ff27000300e00052
:100a500015003b00010028004f01be00000005000a
:100a600000004000818048008502e900fcff3a0058
:100a700009003700f88f420003003c008000eb00c3
:100a80004f01be00000005008100d1000080d300ae
:100a90008502e800fcff3a000300e00002003b0092
:100aa00060001000e08018004f01be00000006004a
:100ab000829fbe000001be00540007000470a70022
:100ac00003f0a10003f8a30015003a006509b10086
:100ad000110032000a0035006928e10003003500ea
:100ae000010028004f01be0000000500000040008a
:100af000818048008502e900fcff3a0006003700cb
:100b0000f88f4200060035008100d1000080d3003c
:100b10008502e800fcff3a004f01be00000006001d
:100b20008000eb004f01be0000000500cf80de001a
:100b3000010037008000eb00829fbe00889fbe004e
:100b40008a9fbe00010578000100e0000400350026
:100b500008003c000000e0002000320005003700e3
:100b600060001000e080180002003b0001f024004b
:100b70001a0037000004be006011b8006b092000a5
:100b80000982cf00020039000882cf000441b00082
:100b9000694252000e00320008003b008281710061
:100ba000610164008904d1000884d3008b05e8004a
:100bb0000442e800f9ff3a00050037000804440049
:100bc00089844c008b05e9000442e900fbff3a00f0
:100bd000230007000af0a70001f0a0004f05be00a7
:100be0004f04be004f01be00000006000004be001e
:100bf000060007000003be000405be000200be00a0
:100c000002000700844f750000000600c70ade00de
:100c1000f107b200f50fb20008003200e1cf420048
:100c2000020032000170a00024000500810f700056
:100c3000010032000408050044000500810f700027
:100c400002003a00140005008502e900000040009f
:100c500081c04800fcff3b000170a000240005009b
:100c600081002000618055000b003d000b0020003a
:100c700061fe2f000100e1001d003400828171003f
:100c8000610164008904d1000884d3000000e800f9
:100c9000faff3a0071002000610064000300700058
:100ca000020060000900320061044400e0844c004e
:100cb0000988a500050032008b05e8006808e100fe
:100cc00002003a008904d1000884d300f20f20000a
:100cd0000258e10005003d00c75ddd00f907b200e4
:100ce0008980750008007800000006000bf82700d6
:100cf0008b007800000005000200be006450e10097
:100d0000050036006420e100020036000968a300f7
:100d100001003a000800be000160a0004f06be00be
:100d20004f05be004f04be004f03be00000006008a
:100d3000f0ff2f00f1ff2700f8ff37000020ef0041
:100d40000220ef00c088a900004006000f0021002b
:100d5000b02e210000018800000000000000eb0020
:100d6000000778000c000900002f78000007eb0056
:100d70005420ef000e2eef001e2eef000000eb00bf
:100d8000a1212100e51d09008018780040a7a900d5
:100d9000a10020009afd0700e0022000303a880000
:100da00044e7a90044c7a9004407a9004427a900b3
:100db0004447a9004467a9004487a90030002000e7
:100dc0000600fc003174200082072000a3092000e7
:100dd000824878008348780080487800113a800083
:100de000618070000600fc00217420006204200075
:100df0007305200082487800834878008048780096
:100e00004427ef00e0022000303a88003000200044
:100e10000d00fc003174200082072000a30920008f
:100e200082487800834878008048780000002000dd
:100e3000217420006204200073052000824878009d
:100e4000834878008048780042a7ae00feff370054
:100e5000813e20006afd070010c0b30086e6b7009f
:100e600090c2b300c4e6b700000220000070880002
:100e7000007025008070880010eea90010cea90037
:100e800010aea900008ea900108ea900000ea900c6
:100e9000002ea900100ea900102ea900c104070001
:100ea000a7050700bc060700a50607000000eb0029
:100eb000c1972100ff000900805878005472ef00ac
:100ec0005572ef003832ef003a32ef000080eb004d
:100ed000c156210007000900801878002232ef0077
:100ee0003632ef004188a90041a8a90041c8a800f6
:100ef00000a1ef00005822001008880004a1a900fa
:100f00000481a80005e1a8000068a9002068a800e5
:100f10001061a8001021a90011e1a80011a1a900e9
:100f200010a1a8001081a8000621ef000a21ef00ff
:100f30000ca1ef000ea1ef004408a9004428a9006d
:100f40004448a9000108a9002108a8002002a9001e
:100f50002022a9002042a90020a2a9002062a90005
:100f60002082a90020e2a9002102a9002122a900d3
:100f7000700720004011880022a2a90022c2a90007
:100f800022e2a90021e2a8002182a9004588a90047
:100f900045a8a80045c8a8002168a8002828a800de
:100fa0002bc8a9002be8a9002c08a9000bc8a90090
:100fb0000be8a9000c08a90001eca90001aca900ec
:100fc000016ca900014ca900012ca900010ca90089
:100fd00000eca900008ca90000aca90000cca9007d
:100fe000000ca900002ca900004ca900006ca9006d
:100ff000202cef00402cef00602cef0000102000b0
:1010000020608800020ca900022ca800024ca90054
:10101000f007200030618800f0072000306288006f
:10102000f007200030638800282cef00482cef00e8
:10103000682cef00001020005060880023eca8000e
:1010400023cca80023aca900238ca900236ca90001
:10105000234ca900232ca900230ca900222ca900b1
:1010600043eca80043cca80043aca900438ca900e2
:10107000436ca900434ca900432ca900430ca900d0
:1010800063eca80063cca80063aca900638ca80043
:10109000636ca900634ca900dabc2a001b3224004f
:1010a00030002c00fa608800fb6088002061880016
:1010b000dabc2a001b32240000002c00fa608800f1
:1010c000fb60880010618800dabc2a001b32240013
:1010d00030002c00fa608800fb60880020628800e5
:1010e000dabc2a001b32240000002c00fa608800c1
:1010f000fb60880010628800dabc2a001b322400e2
:1011000030002c00fa608800fb60880020638800b3
:10111000dabc2a001b32240000002c00fa60880090
:10112000fb60880010638800a80037003f0037008c
:10113000002020000061880000202000006288005c
:101140000020200000638800020ca900022ca800e7
:10115000024ca80004acef0028acef0048acef0054
:1011600068acef00262cef00462cef00662cef0059
:101170000aacef0023eca80023cca90043eca800a4
:1011800043cca90063eca80063cca900dabc2a0018
:101190001b32240030002c00fa608800fb608800bd
:1011a00020618800dabc2a001b32240000002800dd
:1011b000fa608800fb60880010618800dabc2a00b1
:1011c0001b32240030002c00fa608800fb6088008d
:1011d00020628800dabc2a001b32240000002800ac
:1011e000fa608800fb60880010628800dabc2a0080
:1011f0001b32240030002c00fa608800fb6088005d
:1012000020638800dabc2a001b322400000028007a
:10121000fa608800fb6088001063880011eea90066
:1012200011aea900116ea900680037003600370022
:10123000001020000061880000102000006288007b
:101240000010200000638800020ca900022ca800f6
:10125000024ca8000a2cef0000402000206088000b
:10126000282cef005055250040628800a0aa2a00d3
:1012700040638800dabc2a001b32240030002c00b6
:10128000fa608800fb60880020618800dabc2a00d0
:101290001b32240000002c00fa608800fb608800ec
:1012a00010618800dabc2a001b32240030002c00b8
:1012b000fa608800fb60880020628800dabc2a009f
:1012c0001b32240000002c00fa608800fb608800bc
:1012d00010628800dabc2a001b32240030002c0087
:1012e000fa608800fb60880020638800dabc2a006e
:1012f0001b32240000002c00fa608800fb6088008c
:1013000010638800310037003000370000102000e3
:10131000006188000010200000628800020ca90013
:10132000022ca800024ca8000a2cef0004acef002d
:10133000282cef000000240040628800dabc2a005c
:101340001b32240030002c00fa608800fb6088000b
:1013500020618800dabc2a001b32240000002c0027
:10136000fa608800fb60880010618800dabc2a00ff
:101370001b32240030002c00fa608800fb608800db
:1013800020628800dabc2a001b32240000002c00f6
:10139000fa608800fb60880010628800dabc2a00ce
:1013a0001b32240030002c00fa608800fb608800ab
:1013b00020638800dabc2a001b32240000002c00c5
:1013c000fa608800fb60880010638800218ca90007
:1013d000418ca900618ca900216ca900416ca90075
:1013e000616ca900214ca900414ca900614ca900e5
:1013f00020eca80040eca80060eca8003e2cef0018
:101400005e2cef007e2cef0001eca80026013700d7
:10141000ff3ffc004200f8003600f8004400f800ee
:101420008e1f78000e0020000d000900be1f7800fe
:101430003200f8000100fc000068a9000021ef0064
:1014400022928000339280000000200001302400ae
:10145000dffc070096fd07003061880042928000a3
:10146000539280000000200001302400d8fc0700c7
:101470008ffd0700306288006292800073928000c6
:101480000000200001302400d1fc070088fd070087
:10149000306388006672ec006612af00040ea8008c
:1014a0006612ae00040ea900ff3ffc003200f900f6
:1014b000ae0120000d0009004f1778004f0778009b
:1014c0004400f9003600f9004200f9000100fc0078
:1014d00000400600ff3ffc004200f8003600f80024
:1014e0004400f8008e1f78000e0020000d00090057
:1014f000be1f78003200f8000100fc000108a900be
:10150000ff3ffc003200f900ae0120000d00090091
:101510004f1778004f0778004400f9003600f900b3
:101520004200f9000100fc0000400600ff3ffc0003
:101530004200f8003600f8004400f8008e1f7800e2
:101540000e0020000d000900be1f78003200f800d8
:101550000100fc000368a9001421ef00ff3ffc001c
:101560003200f900ae0120000d0009004f1778008d
:101570004f0778004400f9003600f9004200f900f6
:101580000100fc0000400600ff3ffc004200f800a4
:101590003600f8004400f8008e1f78000e0020008e
:1015a0000d000900be1f78003200f8000100fc00a9
:1015b0000388a9001821ef00ff3ffc003200f9006a
:1015c000ae0120000d0009004f1778004f0778008a
:1015d0004400f9003600f9004200f9000100fc0067
:1015e00000400600ff3ffc004200f8003600f80013
:1015f0004400f8008e1f78000e0020000d00090046
:10160000be1f78003200f8000100fc000168a9004c
:101610005472ec0054d2bf008080fb003011800077
:10162000c297210080707900ff3ffc003200f90072
:10163000ae0120000d0009004f1778004f07780019
:101640004400f9003600f9004200f9000100fc00f6
:1016500000400600ff3ffc004200f8003600f800a2
:101660004400f8008e1f78000e0020000d000900d5
:10167000be1f78003200f8000100fc000828a90015
:101680002242ae00000037002222af002222a90031
:10169000ff3ffc003200f900ae0120000d00090000
:1016a0004f1778004f0778004400f9003600f90022
:1016b0004200f9000100fc0000400600ff3ffc0072
:1016c0004200f8003600f8004400f8008e1f780051
:1016d0000e0020000d000900be1f78003200f80047
:1016e0000100fc000188a900ff3ffc003200f90066
:1016f000ae0120000d0009004f1778004f07780059
:101700004400f9003600f9004200f9000100fc0035
:1017100000400600ff3ffc004200f8003600f800e1
:101720004400f8008e1f78000e0020000d00090014
:10173000be1f78003200f8000100fc0001a8a900db
:101740002003a900ff3ffc003200f900ae01200099
:101750000d0009004f1778004f0778004400f9008a
:101760003600f9004200f9000100fc0000400600cc
:10177000ff3ffc004200f8003600f8004400f8008b
:101780008e1f78000e0020000d000900be1f78009b
:101790003200f8000100fc000bc8a900ff3ffc006c
:1017a0003200f900ae0120000d0009004f1778004b
:1017b0004f0778004400f9003600f9004200f900b4
:1017c0000100fc0000400600ff3ffc004200f80062
:1017d0003600f8004400f8008e1f78000e0020004c
:1017e0000d000900be1f78003200f8000100fc0067
:1017f0000be8a900ff3ffc003200f900ae01200019
:101800000d0009004f1778004f0778004400f900d9
:101810003600f9004200f9000100fc00004006001b
:10182000ff3ffc004200f8003600f8004400f800da
:101830008e1f78000e0020000d000900be1f7800ea
:101840003200f8000100fc000c08a900ff3ffc007a
:101850003200f900ae0120000d0009004f1778009a
:101860004f0778004400f9003600f9004200f90003
:101870000100fc000040060055d2bf005452e300b6
:10188000070032005572ec0055d2bf000080fb000b
:10189000c197210060c0780056f2b7000100370000
:1018a00056f2ef000000060050088000d09188003a
:1018b00030088000c0918800efff070060ceb300c1
:1018c0005652b50006003900e0cfb3005652b500bd
:1018d00001003900010037005772ef00490137005d
:1018e00056f2ae00370037005772ef0050c8b30011
:1018f0005652e30005003a0056d2bf0057f2b70037
:1019000058f2ef0059f2ef002d00370050c9b30034
:101910005652e30005003a0056d2bf0057f2b70016
:101920005af2ef005bf2ef002500370050cab30017
:101930005652e30005003a0056d2bf0057f2b700f6
:101940005cf2ef005df2ef001d00370050cbb300fa
:101950005652e30005003a0056d2bf0057f2b700d6
:101960005ef2ef005ff2ef001500370050ccb300dd
:101970005652e30004003a0056d2bf0057f2b700b7
:1019800060f2ef000e00370050cdb3005652e30076
:1019900004003a0056d2bf0057f2b70061f2ef00e0
:1019a0000700370050ceb3005652e30004003a005f
:1019b00056d2bf0057f2b70062f2ef0063f2ef00b9
:1019c000100137005752e20002003a000d013700c3
:1019d0000c01370050c8b3005752e30049003a00e9
:1019e00000e0ef005852e30003003a0056d2bf0077
:1019f00058f2b7004200370056d2bf0059f2b70084
:101a000090c1b3005852e3002e003a005952e20050
:101a100013003a0014cea9006672ef0005e1a90098
:101a2000f007200030618800f00720003062880055
:101a3000f0072000306388003032ef003412a90034
:101a40002212ae00040037006cb5ef006eb5ef0057
:101a50006512a8002212a900140ea9001800370070
:101a6000022eae00160037003412a80005e1a800cf
:101a70000200210059d2bf000080fb000200b80024
:101a80000001be0062ab880073ab880062ab8000cf
:101a900073ab8000c0918000d191800002004000b3
:101aa000838048000001be0062ab880073ab8800f1
:101ab0002212a8006512a800140ea900142ea80076
:101ac0000e00370080c7b3005852e30002003a000e
:101ad00014aea9000900370090c7b3005852e300c4
:101ae00002003a00048ea90004003700a0c7b3002a
:101af0005852e30001003a00148ea90058f2ef009a
:101b0000c000370050c9b3005752e30070003a00dc
:101b100000e0ef005a52e30003003a0056d2bf0043
:101b20005af2b7006900370056d2bf005bf2b70027
:101b30005b52e20025003a0090c1b3005a52e30024
:101b400013003a0014cea9006672ef0005e1a90067
:101b5000f007200030618800f00720003062880024
:101b6000f0072000306388003032ef003412a90003
:101b70002212ae00040037006cb5ef006eb5ef0026
:101b80006512a8002212a900140ea9000e00370049
:101b900080c7b3005a52e30002003a0014aea90015
:101ba0000900370090c7b3005a52e30002003a0020
:101bb000048ea90004003700a0c7b3005a52e30006
:101bc00001003a00148ea9003f00370090c1b30015
:101bd0005a52e30022003a005bd2bf006af2b7001b
:101be000022eae001a00370014cea8006ad2bf0041
:101bf0000080fb0000004000c146210060807800aa
:101c00001008880005e1a8000068a9002068a80065
:101c10006672ef005bd2bf000080fb00c1a721000d
:101c200060c078000080fb00809188003412a90019
:101c30002212ae00040037006cb5ef006eb5ef0065
:101c40006512a8002212a900140ea8000300370094
:101c500014cea900140ea9003032ef001a0037008c
:101c600080c7b3005a52e30006003a00022eae00cd
:101c70000200370014aea8000100370014aea9001e
:101c80001100370090c7b3005a52e30006003a0033
:101c9000022eae0002003700048ea80001003700bb
:101ca000048ea90008003700a0c7b3005a52e30011
:101cb00005003a00022eae0002003700148ea80084
:101cc00001003700148ea9005af2ef004d003700d2
:101cd00050cab3005752e3001c003a0000e0ef0086
:101ce0005c52e30003003a0056d2bf005cf2b7003a
:101cf0001500370056d2bf005df2b70090c1b300a7
:101d00005c52e3000f003a0012ceae000d00370027
:101d10006672ef005dd2bf000080fb00c1a721000a
:101d200060c078000080fb00809188005dd2bf0019
:101d30000080fb0000004000c14621006080780068
:101d4000100888005cf2ef002e00370050cbb30083
:101d50005752e3000b003a0000e0ef005e52e30050
:101d600003003a0056d2bf005ef2b700040037000d
:101d700056d2bf005ff2b700e50007005ef2ef0049
:101d80002000370050ccb3005752e30007003a0060
:101d900000e0ef006052e30003003a0056d2bf00bb
:101da00060f2b70060f2ef001600370050cdb300cc
:101db0005752e30007003a0000e0ef006152e300f1
:101dc00003003a0056d2bf0061f2b70061f2ef00a3
:101dd0000c00370050ceb3005752e30009003a0020
:101de00000e0ef006252e30003003a0056d2bf0069
:101df00062f2b7000300370056d2bf0063f2b700ab
:101e000062f2ef006512af00a400070040c0b3000b
:101e10006452b50038003100c2918000d391800037
:101e20000092800011928000800f5100818f590034
:101e30002500390043f2a8006452e20010003a0085
:101e400014cea9006672ef0005e1a900f00720009a
:101e500030618800f007200030628800f007200021
:101e6000306388003032ef006cb5ef006eb5ef00e4
:101e70003412a9002212a900142ea9001100370063
:101e800010c0b3006452e30003003a0070b5ef00e5
:101e900072b5ef000b00370020c0b3006452e300be
:101ea00003003a0074b5ef0076b5ef000500370087
:101eb00030c0b3006452e30002003a0078b5ef008e
:101ec0007ab5ef00750007003bf2ae00090037005d
:101ed0000621ef000a21ef003832ef003a32ef001e
:101ee0000080eb00c156210007000900801878002f
:101ef0006dfe3700040037003bf2ae0002003700f1
:101f00000621ef000a21ef0067d2bf006652e3000e
:101f10005d0032003412af002d00370066d2bf00e2
:101f20000080fb00c200dd00c0572100008040009f
:101f30001000be000001be0080918000fbfa070087
:101f400081fa0700209288003192880066d2bf0093
:101f50005041b00068f2b70068d2bf000080fb00bb
:101f6000c200dd00c0572100008040001000be000c
:101f70000001be0080918000ecfa070072fa0700b1
:101f8000409288005192880066d2bf00b042b000f3
:101f900069f2b70069d2bf000080fb00c200dd001b
:101fa000c0572100008040001000be000001be00ac
:101fb00080918000ddfa070063fa070060928800d4
:101fc0007192880066d2bf0067f2b7002e0037001a
:101fd0002212ae002a00370066d2bf000080fb004c
:101fe000c200dd00c0572100008040001000be008c
:101ff0000001be0080918000ccfa070052fa070071
:10200000209288003192880050c1b3006652b5001a
:1020100068f2b70068d2bf000080fb00c200dd009c
:10202000c0572100008040001000be000001be002b
:1020300080918000bdfa070043fa070040928800b3
:1020400051928800b0c2b3006652b50069f2b70081
:1020500069d2bf000080fb00c200dd00c057210034
:10206000008040001000be000001be008091800092
:10207000aefa070034fa0700609288007192880077
:1020800066d2bf0067f2b7003a32af0014eea80084
:102090003a32ae0014eea90003fe370064f2ef00fe
:1020a00043f2a8002032ef0000918000c200dd0062
:1020b000c0562100008040001000be000001be009c
:1020c0000092800011928000800f5100818f590092
:1020d0000900310000918000c200dd00c0562100df
:1020e000008040001000be0000928800119288001d
:1020f00020d2bf0064f2b7002032ec0001918000d2
:10210000e48f5000e8ff3a006512a90000000600c5
:1021100020c4b3005e52e30019003a005f52e200af
:1021200015003a002032ef0001918000e38f50004b
:1021300009003e0000918000c200dd00c056210071
:1021400000814000f0ff2f00f1ff2f000089be004a
:102150002032ec00f4ff39006512a80014cea9006b
:1021600014aea900048ea900148ea900042ea900a3
:10217000142ea90001003700042ea8000700370024
:10218000b0c7b3005e52e30004003a0014cea900c9
:1021900014aea900048ea900148ea9005ef2ef000f
:1021a000000006006cb3ef00101a2f00709b88002f
:1021b00010412e00809b880040742d00909b880069
:1021c000f0b22c00a09b880070fc2b00b09b880014
:1021d00030502b00c09b8800a0ad2a00d09b880007
:1021e00030142a00e09b880060832900f09b88005f
:1021f000b0fa2800009c8800a0792800109c880074
:10220000c00020000091880001918000f78f5000ed
:102210000e003e00c00020002012b500000678002d
:102220000c064600c036210060007e004100de0042
:10223000029180004111dd00c13621000101410001
:10224000000978002032ec00efff39008001200007
:10225000009188000191800030022000808f5000a2
:102260000e003e00800120002012b500000678001c
:102270000c064600c036210060007e004200de00f1
:10228000029180004111dd00c136210001014100b1
:10229000000978002032ec00eeff390040022000f7
:1022a0000091880001918000f0022000808f500092
:1022b0000e003e00400220002012b500000678000b
:1022c0000c064600c036210060007e004300de00a0
:1022d000029180004111dd00c13621000101410061
:1022e000000978002032ec00eeff390000032000e6
:1022f0000091880001918000b0032000808f500081
:102300000e003e00000320002012b50000067800f9
:102310000c064600c036210060007e004400de004e
:10232000029180004111dd00c13621000101410010
:10233000000978002032ec00eeff3900c0032000d5
:10234000009188000191800070042000808f50006f
:102350000e003e00c00320002012b50000067800e9
:102360000c064600c036210060007e004500de00fd
:10237000029180004111dd00c136210001014100c0
:10238000000978002032ec00eeff390080042000c4
:10239000009188000191800030052000808f50005e
:1023a0000e003e00800420002012b50000067800d8
:1023b0000c064600c036210060007e004600de00ac
:1023c000029180004111dd00c13621000101410070
:1023d000000978002032ec00eeff3900007a21007d
:1023e000a0a08800f0732100b0a08800f06d21004b
:1023f000c0a0880000682100d0a0880040622100b1
:10240000e0a08800805c2100f0a08800e056210058
:1024100000a188006051210010a18800f04b21002c
:1024200020a188009046210030a188005041210061
:1024300040a18800203c210050a1880010372100d5
:1024400060a188001032210070a18800202d210099
:1024500080a188004028210090a1880080232100cd
:10246000a0a18800d01e2100b0a18800301a210050
:10247000c0a18800a0152100d0a188002011210052
:10248000e0a18800c00c2100f0a1880070082100a4
:1024900000a288002004210010a28800f0ff200084
:1024a00020a28800d0fb200030a28800c0f72000c6
:1024b00040a28800d0f3200050a28800e0ef200066
:1024c00060a2880000ec200070a2880030e82000a4
:1024d00080a2880070e4200090a28800c0e0200064
:1024e000a0a2880020dd2000b0a2880090d92000a2
:1024f000c0a2880010d62000d0a28800a0d2200060
:10250000e0a2880040cf2000f0a28800e0cb2000ad
:1025100000a38800a0c8200010a3880060c5200088
:1025200020a3880030c2200030a3880010bf200004
:1025300040a3880000bc200050a3880000000600d3
:102540006cb2ef00a0c7250070938800509825005a
:10255000809388004081250090938800906a250030
:10256000a093880030542500b0938800303e2500a9
:10257000c093880090282500d09388005013250030
:10258000e093880060fe2400f0938800c0e92400f6
:102590000094880080d524001094880090c1240005
:1025a00020948800f0ad240030948800a09a240084
:1025b00040948800a087240050948800f074240080
:1025c00060948800906224007094880080502400f9
:1025d00080948800b03e240090948800302d240020
:1025e000a0948800f01b2400b0948800000b240005
:1025f000c094880050fa2300d0948800e0e92300ba
:10260000e0948800c0d92300f0948800e0c923003a
:102610000095880040ba230010958800e0aa2300a6
:1026200020958800c09b230030958800e08c230013
:1026300040958800307e230050958800d06f23009d
:1026400060958800a061230070958800b053230036
:1026500080958800f045230090958800703823000d
:10266000a0958800202b2300b0958800101e230021
:10267000c095880040112300d09588009004230065
:10268000e095880020f82200f0958800e0eb220019
:1026900000968800d0df220010968800f0d3220038
:1026a0002096880050c8220030968800d0bc2200b6
:1026b0004096880080b122005096880070a62200c3
:1026c00060968800809b220070968800c09022004f
:1026d000809688002086220090968800c07b220089
:1026e000a096880080712200b09688006067220062
:1026f000c0968800805d2200d0968800c0532200da
:10270000e0968800204a2200f0968800b04022001f
:10271000009788006037220010978800402e220022
:10272000209788004025220030978800601c2200f6
:1027300040978800b013220050978800200b220099
:1027400060978800b00222007097880060fa21002c
:102750008097880040f221009097880030ea21009d
:10276000a097880050e22100b097880090da2100fd
:10277000c0978800e0d22100d097880060cb21006c
:10278000e0978800f0c32100f0978800b0bc2100da
:102790000098880080b521001098880080ae210044
:1027a0002098880090a7210030988800b0a02100d0
:1027b00040988800009a210050988800609321007a
:1027c00060988800e08c2100709888008086210045
:1027d000809888003080210090988800007a21003d
:1027e000a0988800f0732100b0988800f06d210057
:1027f000c098880000682100d098880040622100bd
:10280000e0988800805c2100f0988800e056210064
:10281000009988006051210010998800f04b210038
:10282000209988009046210030998800504121006d
:1028300040998800203c21005099880010372100e1
:10284000609988001032210070998800202d2100a5
:1028500080998800402821009099880080232100d9
:10286000a0998800d01e2100b0998800301a21005c
:10287000c0998800a0152100d0998800201121005e
:10288000e0998800c00c2100f099880070082100b0
:10289000009a880020042100109a8800f0ff200090
:1028a000209a8800d0fb2000309a8800c0f72000d2
:1028b000409a8800d0f32000509a8800e0ef200072
:1028c000609a880000ec2000709a880030e82000b0
:1028d000809a880070e42000909a8800c0e0200070
:1028e000a09a880020dd2000b09a880090d92000ae
:1028f000c09a880010d62000d09a8800a0d220006c
:10290000e09a880040cf2000f09a8800e0cb2000b9
:10291000009b8800a0c82000109b880060c5200094
:10292000209b880030c22000309b880010bf200010
:10293000409b880000bc2000509b880000000600df
:1029400090dc230090928800b0fd200080928800e7
:102950002032ef0021f2bf000e003a008292800088
:10296000939280000091800072f80700f6f707004c
:10297000bcf607000001be0000918000c200dd002f
:10298000c0572100008040000288be002032ec00c9
:10299000f0ff390000000600c012200050ab880094
:1029a0001013200040ab88006013200030ab88007b
:1029b000b013200020ab88000014200010ab88006a
:1029c0005014200000ab8800b0142000f0aa88004a
:1029d00000152000e0aa880060152000d0aa880019
:1029e000b0152000c0aa880010162000b0aa8800e8
:1029f00070162000a0aa8800d016200090aa880097
:102a00003017200080aa88009017200070aa880044
:102a1000f017200060aa88005018200050aa8800f3
:102a2000b018200040aa88002019200030aa880091
:102a30008019200020aa8800f019200010aa880020
:102a4000601a200000aa8800d01a2000f0a988008f
:102a5000401b2000e0a98800b01b2000d0a98800fe
:102a6000201c2000c0a98800a01c2000b0a988005c
:102a7000101d2000a0a98800901d200090a98800aa
:102a8000101e200080a98800801e200070a98800e8
:102a9000001f200060a98800901f200050a9880016
:102aa0001020200040a988009020200030a9880034
:102ab0002021200020a98800a021200010a9880042
:102ac0003022200000a98800c0222000f0a8880041
:102ad00050232000e0a88800f0232000d0a8880020
:102ae00080242000c0a8880020252000b0a88800ed
:102af000b0252000a0a888005026200090a88800bb
:102b0000f026200080a888009027200070a8880068
:102b10004028200060a88800e028200050a88800f5
:102b20009029200040a88800402a200030a8880072
:102b3000f02a200020a88800a02b200010a88800e0
:102b4000602c200000a88800102d2000f0a788002d
:102b5000d02d2000e0a78800902e2000d0a788006c
:102b6000502f2000c0a7880020302000b0a7880088
:102b7000e0302000a0a78800b031200090a7880096
:102b80008032200080a788005033200070a7880082
:102b90003034200060a788001035200050a788003e
:102ba000e035200040a78800d036200030a78800fc
:102bb000b037200020a788009038200010a7880098
:102bc0008039200000a78800703a2000f0a6880015
:102bd000703b2000e0a68800603c2000d0a6880062
:102be000603d2000c0a68800603e2000b0a688009e
:102bf000703f2000a0a688007040200090a68800aa
:102c00008041200080a688009042200070a68800a5
:102c1000b043200060a68800c044200050a6880071
:102c2000e045200040a688001047200030a688001c
:102c30003048200020a688006049200010a68800a7
:102c4000a04a200000a68800d04b2000f0a58800f4
:102c5000104d2000e0a58800504e2000d0a588002f
:102c6000a04f2000c0a58800f0502000b0a588002b
:102c700040522000a0a588009053200090a5880015
:102c8000f054200080a588005056200070a58800d0
:102c9000c057200060a588003059200050a588004a
:102ca000a05a200040a58800205c200030a58800a4
:102cb000a05d200020a58800305f200010a58800be
:102cc000c060200000a5880050622000f0a48800a9
:102cd000f0632000e0a4880090652000d0a4880064
:102ce00040672000c0a48800f0682000b0a48800dd
:102cf000a06a2000a0a48800606c200090a4880036
:102d0000306e200080a48800f06f200070a488003e
:102d1000d071200060a48800b073200050a4880007
:102d20009075200040a488008077200030a488009f
:102d30007079200020a48800707b200010a48800f7
:102d4000707d200000a48800807f2000f0a3880010
:102d5000a0812000e0a38800c0832000d0a38800c9
:102d6000e0852000c0a3880010882000b0a3880060
:102d7000508a2000a0a38800908c200090a3880097
:102d8000e08e200080a388003091200070a388008e
:102d90009093200060a3880000c1b3007cfab700c4
:102da00000c1b3007dfab70010c1b3007efab700ce
:102db00010c1b3007ffab70010c1b30080fab700aa
:102dc00010c1b30081fab70020c1b30082fab70086
:102dd00020c1b30083fab70020c1b30084fab70062
:102de00030c1b30085fab70030c1b30086fab7002e
:102df00030c1b30087fab70040c1b30088fab7000a
:102e000040c1b30089fab70040c1b3008afab700e5
:102e100040c1b3008bfab70050c1b3008cfab700c1
:102e200050c1b3008dfab70050c1b3008efab7009d
:102e300060c1b3008ffab70060c1b30090fab70069
:102e400060c1b30091fab70070c1b30092fab70045
:102e500070c1b30093fab70080c1b30094fab70011
:102e600080c1b30095fab70080c1b30096fab700ed
:102e700090c1b30097fab70090c1b30098fab700b9
:102e8000a0c1b30099fab700a0c1b3009afab70085
:102e9000b0c1b3009bfab700b0c1b3009cfab70051
:102ea000b0c1b3009dfab700c0c1b3009efab7002d
:102eb000c0c1b3009ffab700d0c1b300a0fab700f9
:102ec000d0c1b300a1fab700e0c1b300a2fab700c5
:102ed000e0c1b300a3fab700f0c1b300a4fab70091
:102ee000f0c1b300a5fab70000c2b300a6fab7005c
:102ef00000c2b300a7fab70010c2b300a8fab70027
:102f000010c2b300a9fab70020c2b300aafab700f2
:102f100020c2b300abfab70030c2b300acfab700be
:102f200040c2b300adfab70040c2b300aefab7007a
:102f300040c2b300affab70050c2b300b0fab70056
:102f400060c2b300b1fab70060c2b300b2fab70012
:102f500070c2b300b3fab70080c2b300b4fab700ce
:102f600080c2b300b5fab70090c2b300b6fab7009a
:102f7000a0c2b300b7fab700b0c2b300b8fab70046
:102f8000b0c2b300b9fab700c0c2b300bafab70012
:102f9000c0c2b300bbfab700d0c2b300bcfab700de
:102fa000e0c2b300bdfab700f0c2b300befab7008a
:102fb000f0c2b300bffab70000c3b300c0fab70055
:102fc00010c3b300c1fab70020c3b300c2fab70000
:102fd00030c3b300c3fab70040c3b300c4fab700ac
:102fe00040c3b300c5fab70050c3b300c6fab70078
:102ff00060c3b300c7fab70070c3b300c8fab70024
:1030000080c3b300c9fab70090c3b300cafab700cf
:10301000a0c3b300cbfab700b0c3b300ccfab7007b
:10302000c0c3b300cdfab700c0c3b300cefab70037
:10303000e0c3b300cffab700f0c3b300d0fab700d3
:1030400000c4b300d1fab70010c4b300d2fab7007d
:1030500020c4b300d3fab70030c4b300d4fab70029
:1030600040c4b300d5fab70050c4b300d6fab700d5
:1030700060c4b300d7fab70070c4b300d8fab70081
:1030800090c4b300d9fab700a0c4b300dafab7000d
:10309000b0c4b300dbfab700c0c4b300dcfab700b9
:1030a000d0c4b300ddfab700f0c4b300defab70055
:1030b00000c5b300dffab70010c5b300e0fab700ef
:1030c00030c5b300e1fab70040c5b300e2fab7007b
:1030d00050c5b300e3fab70070c5b300e4fab70017
:1030e00080c5b300e5fab700a0c5b300e6fab700a3
:1030f000b0c5b300e7fab700c0c5b300e8fab7003f
:10310000e0c5b300e9fab70000c6b300eafab700b9
:1031100010c6b300ebfab70030c6b300ecfab70044
:1031200040c6b300edfab70060c6b300eefab700d0
:1031300080c6b300effab70090c6b300f0fab7004c
:10314000b0c6b300f1fab700d0c6b300f2fab700c8
:10315000f0c6b300f3fab70000c7b300f4fab70043
:1031600020c7b300f5fab70040c7b300f6fab700be
:1031700060c7b300f7fab70080c7b300f8fab7002a
:10318000a0c7b300f9fab700c0c7b300fafab70096
:10319000e0c7b300fbfab70000000600ffff3700ee
:020000040000fa
:1031a0001a1200000600000080000000201200003b
:1031b0001800000080000000381200001c00000011
:1031c0008000000054120000180000008000000081
:1031d0006c12000000030000800000006c1500006d
:1031e00010040000800000007c1900008001000035
:0831f000800000000000000057
:00000001FF
